:020000040000FA
:020000006B296A
:06000A00820720343434AB
:100010002E3433342034723465345634203465340D
:1000200074346934753473342034743473346534FF
:10003000743420344C3445342D34433449345034F2
:10004000820720347334443445344C3482072034DE
:1000500073346E346F3474347434753442348207BC
:100060002034733465346C34643464346134503413
:1000700082072034723465346B34613465347034F3
:100080005334820720347234653464346F346334FB
:100090006E34453482072034743469346D347334DB
:1000A0006E3461347234543482072034533444340F
:1000B000443408307C20362100307C203621080072
:1000C00008307C20362108307C20362108000030A2
:1000D0007C2001307C203621080000307C20073055
:1000E0007C203E210800EF3986001038860032213E
:1000F000EF398600322108000F39732008000F39CC
:100100003038B700F039B800B80CB80CB80CB80CDF
:1001100038084038732037080F39403873203E21A3
:1001200008001230B6003621B60B932803307C202D
:10013000362103307C203E2103307C203E210230DA
:100140007C20362102307C2008307C203621003093
:100150007C2008307C20362100307C2001307C203F
:10016000362100307C2006307C20362100307C2077
:100170000C307C2036210800672060206D2019306B
:10018000B6004621360805208120B60BC128522131
:1001900000307C2004307C203E216720080067204E
:1001A0000430B600360820208120B60BD228080083
:1001B00067200730B600360826208120B60BDB28E2
:1001C000080067200730B60036082F208120B60BC4
:1001D000E428080067200730B60036083820812060
:1001E000B60BED28080067200730B600360841201E
:1001F0008120B60BF628080067200830B6003608C4
:100200004A208120B60BFF28080067200330B60083
:10021000360854208120B60B082908000330BE00A0
:100220001030BF00BF0B1229BE0B10290800503040
:10023000C00005150E2105110E21C00B192905114D
:100240000800B300672017215430812065308120D9
:100250007330812074308120203081203308812048
:100260005221172900000000000008001830BB00D0
:10027000BC00BC0B3929BB0B382908000430B9007D
:10028000BA00BA0B4129B90B402908005030B90017
:100290003621B90B48290800BE0B0800BF0B080027
:1002A000C00308000830B6004621B60B54290800E8
:1002B000612161216121612161216121612161212E
:1002C0000800FF30CE006429FF30CF00CF0B662935
:1002D000CE0B642908000030B2000030831686007F
:1002E0008312203086001B30831685008312043071
:1002F00085009120BC2031302121CF20982132303F
:100300002121D820AF2133302121E120C9213430EF
:100310002121EA20F02135302121F3201A22363024
:100320002121FC20D222373021210521DD227B2909
:100330000230B2000E30860052210C30860052216D
:100340000A30860052210630860052210E30860087
:100350005221003086005221B20B9A2908000A303F
:10036000C000FF30BE00BF00831605158312B10127
:10037000051AB115851931150519B1143108860012
:100380004C214008031DB72983160511831205115E
:1003900008000A30C000FF30BE00BF00B10185195F
:1003A000B115051AB114310886004C214008031D0F
:1003B000CE2908000830BF00BF0BDC29BE0BDA29AC
:1003C00008000430BD0005153208BE00DA21051111
:1003D0003208BE00DA21BD0BE329C00BE129080079
:1003E0003B30C0004430B200E1214230C0003D301B
:1003F000B200E1214A30C0003630B200E1214F3076
:10040000C0003330B200E1215930C0002D30B200BD
:10041000E1216430C0002830B200E1216F30C0001B
:100420002430B200E1217630C0002230B200E12158
:10043000051108008030C500831605148514831249
:100440000A30C000FF30BE00BF009122C100C200D0
:100450005D2246080319502AB301B401B5014508CD
:10046000C400643003144402031C392AB30AC400D4
:10047000312A0A3003144402031C412AB40AC4007E
:10048000392A013003144402031C492AB50AC40066
:10049000412A672033087F2034087F2035087F20D9
:1004A000861106118610411886150615C118861486
:1004B0004E214008031D282A08009122C100C20DC8
:1004C000C20D420841040F39C4004108C200023085
:1004D00044060319892A0B3044060319892A0D3072
:1004E00044060319892A043044060319892A013075
:1004F000440603198D2A0730440603198D2A0E304D
:10050000440603198D2A0830440603198D2AC601B2
:100510000800C50A0130C6000800C5030130C60046
:1005200008000508C3000330C305A92203300505F0
:100530004306031D912AA922033005054306031D26
:10054000912AA922033005054306031D912A430879
:100550000800362108001430B9003621B90BAD2A45
:10056000080006118617AB2206158613AB22080079
:1005700006118617AB22AB22AB2206158613AB22DF
:100580000800AB22AB22AB220800B822C122B12264
:10059000C122B122B122B122C122B822C122C1227C
:1005A000C12208008615061586145221C522C522CF
:1005B000C522C522C522C52208000330B200023080
:1005C000C700BC30C8000530C9001230CA00003076
:1005D000CB0012230E308604FD3086055821C7302B
:1005E000C7006330C8000630C9001230CA000030AE
:1005F000CB0012230E308604FB30860558218D3047
:10060000C7000B30C8000730C9001230CA000030E4
:10061000CB0012230E308604F73086055821B20B2A
:10062000DF2A0800473084000008CD000830CC00E5
:10063000CD0C031C1F2B861506150611222B8611C7
:1006400006150611CC0B182B840A4C300402031C2F
:08065000142B86178613080025
:02400E00F13F80
:00000001FF
